:020000002C28AA
:1000080009008A0182002F344334313446343234B3
:10001800413400342F34433431344634323442349A
:1000280000348A012808A80A82002F341C340034BE
:1000380046341F3400343234223400345234B92860
:100048005434B028563476280D346D2800340034E2
:100058008316263085000830810000309000063075
:100068009F00831216309800073099000516FA3061
:10007800CC210512A0161630D700A001A1018512C7
:100088000530AB00AE006400851E5628B20F472825
:10009800B30A3308013A03197E203308813A031959
:1000A8009720472857211930A8006C21B100152046
:1000B800003A03196728310603196428A80A5B283F
:1000C8001520A80059281520003A031D47283F305D
:1000D800792171207920032147280D307929223090
:1000E80071205828683040216D2805160A30CC2127
:1000F800051208000230C720A3002D06031D922810
:10010800AB0B080023082C06031992282308AC001F
:1001180092200730E8202C0840216D282308AD00E4
:100128000530AB0008000130C720A3003006031DCE
:10013800AB28AE0B080023082F060319AB282308A9
:10014800AF00AB200E30E8202F0840216D2823088F
:10015800B0000530AE0008000230C7204021203032
:1001680079210130C72040216D280230C720C120E5
:10017800FA30CC21A01FB9286D28402120307921E0
:100188002030792108000514CC200510BA3E08005B
:100198000339A3000310A30DA30D23089F001F1408
:1001A800DA219F149F18D6281E080800DC000530A5
:1001B800DB005C08E520201A08007120DB0BDD2835
:1001C8000800E8200E210800DE00FF20BB01851E84
:1001D800E928D821BB0BEB28851EE9288316851250
:1001E80083125E08DE0A0520A300003A03190800FE
:1001F80023087921F52803213F39013EDF295708D3
:10020800D8075808D9070310D90C0318D917590863
:10021800D7070800D10120126430DD00DA219721C8
:10022800A30020181A29DD0B1229080051080A3AE0
:1002380003190E2951083D3E840023088000D10A85
:100248000D3A031D1029D10120160800B6016C21B2
:10025800A3003030A302031C3E290A3023020318EE
:100268003E290310B60D3608B60DB60DB60723089D
:10027800B6072B2936080800A011A40064304821CD
:100288000A304821A0150130A5003030A900250802
:10029800A402031C5229A90AA0154C29A40729085D
:1002A800A01979210800D1019721201C5829640040
:1002B800A3005108123A031947283D305107D10AC3
:1002C8008400230880000D3A031D5829D101080035
:1002D8003D305107D10A840000080800FF30B907F3
:1002E800031CBA073A0839040800B6008512013021
:1002F800CC2104308B2102308B210830B900013029
:10030800B60D031803308B21B90B83290800A3000D
:10031800DA21831685128312DA21A30B902983161A
:10032800851683120800A0102010851A0800AF2136
:10033800AF21A2000830B900B601AF210319AD29D9
:10034800A3002208A302B60DB90BA1293608201470
:100358000800A0140800A301A30A0319080000005C
:100368000000000000000000000000000000851AE6
:10037800B029A301A30A0319080000000000000027
:1003880000000000000000002308851EBE290800A8
:10039800B800A013DE21851EA017B80BCE290800CF
:1003A8000130DF290230DF290530DF290A30DF2953
:1003B8003230DF296430B700000000000000000080
:0C03C800000000000000B70BE029080056
:02400E00E4309C
:00000001FF
